:020000021000EC
:10E000000C9446F00C9466F00C9466F00C9466F058
:10E010000C9466F00C9466F00C9466F00C9466F028
:10E020000C9466F00C9466F00C9466F00C9466F018
:10E030000C9466F00C9466F00C9466F00C9466F008
:10E040000C9466F00C9466F00C9466F00C9466F0F8
:10E050000C9466F00C9466F00C9466F00C9466F0E8
:10E060000C9466F00C9466F00C9466F00C9466F0D8
:10E070000C9466F00C9466F00C9466F00C9466F0C8
:10E080000C9466F00C9466F00C9466F011241FBE9C
:10E09000CFEFD0E1DEBFCDBF11E0A0E0B1E0E8EA14
:10E0A000F0EF01E00BBF02C007900D92A634B1075C
:10E0B000D9F71BBE14E0A6E4B1E001C01D92A43361
:10E0C000B107E1F70E94A9F30C9452F80C9400F008
:10E0D0009C01E199FECF3FBB2EBBE09A8DB3089522
:10E0E0009C01E199FECF3FBB2EBB6DBB0FB6F894F0
:10E0F000E29AE19A0FBE0895E0E0F0E009950895F4
:10E10000E4E6F0E0808181608083119A189A8B9A0E
:10E11000929A0895909128049F5F909328042091EB
:10E120000E03222331F490FF06C0809165008E7F9C
:10E1300005C0213029F480916500816080936500DD
:10E140009A3068F010922804222311F010923304C0
:10E15000809133048A3018F48F5F809333040895DC
:10E160009091460180912504981710F00CC0A89555
:10E1700080919B0085FFFBCFE92FF0E0EA51FD4F36
:10E18000808180939C009F5F909346010895309119
:10E190009C0080912404882309F050C006B600FE3C
:10E1A00006C080911303813011F410921303809103
:10E1B0001303882371F43A32E9F586B7816086BF8C
:10E1C00012BE109223043093220481E08093130343
:10E1D0000895813079F5909123049F5F90932304F3
:10E1E0009D3810F010921303E92FF0E0E35BFD4F30
:10E1F000308320912204230F20932204933041F492
:10E20000832F8C5F8093E3028D3810F010921303FC
:10E210008091E302981771F4822F831B809322046C
:10E22000381741F480911303813021F48093240442
:10E230001092130386B7816086BF12BE0895809145
:10E24000E9028B5F80932504E6EEF2E090E08150D6
:10E25000282F30E02E0F3F1F02C08191980FE21748
:10E26000F307D9F7908381E08093460101C0A89518
:10E2700080919B0085FFFBCF8091E60280939C00FC
:10E280000895EF92FF920F931F93CF93DF93209106
:10E2900014033091150340911603509117032093F6
:10E2A000290430932A0440932B0450932C0480912A
:10E2B0000F0390911003A0911103B091120328173E
:10E2C00039074A075B0791F1E0902D04F0902E0486
:10E2D00000912F0410913004C4E1D3E020E030E03D
:10E2E000C90163E070E00E9407F84C81892B21F09E
:10E2F000842F8F5F821B03C0842F8250820FE80E11
:10E30000F11C011D111DF901E75BFE4F80832F5F9A
:10E310003F4F219681E02030380711F7E0922D041D
:10E32000F0922E0400932F0410933004DF91CF91CC
:10E330001F910F91FF90EF900895EF92FF920F932E
:10E340001F93CF93DF937B018C01A8957FB7E19951
:10E35000FECF83E0F70100935B0080936800E895AF
:10E360008091680080FDFCCFC9E4D1E0A80197014D
:10E3700061E0B981A0E08881FD01E80FF11DCF01C6
:10E380000C01F90140935B0060936800E89511244B
:10E3900022962E5F3F4F4F4F5F4FF2E0C934DF07A9
:10E3A00041F785E0F70100935B0080936800E895F2
:10E3B0008091680080FDFCCF81E180936800E89542
:10E3C0007FBFDF91CF911F910F91FF90EF90089544
:10E3D000A895E199FECF82E090E09FBB8EBB1DBA6D
:10E3E0000FB6F894E29AE19A0FBE84E090E060E004
:10E3F00070E040E750EF0E9451F586E090E060E069
:10E4000070E040E750EF0E9451F588E090E060E056
:10E4100070E040E750EF0E9451F5E199FECF8AE0AD
:10E4200090E09FBB8EBB81E08DBB0FB6F894E29A63
:10E43000E19A0FBEA8950895DF92EF92FF920F9395
:10E440001F93D0904E02E090E50280914F028E150E
:10E4500009F079C1F090510281E0F816C9F5809178
:10E460005202813019F4F0920E0302C010920E0392
:10E4700090910E03913009F082C08AE28093E60207
:10E48000E092E702D092E80289E08093E90290935B
:10E49000EA029093EB028AE090E09093ED02809381
:10E4A000EC0280E091E09093EF028093EE02809185
:10E4B0002604909127049093F1028093F0028091BA
:10E4C0003104909132049093F3028093F20239C1A7
:10E4D00092E0F91661F480910E03813031F480915D
:10E4E00052028093E50210920E0390E048C090E043
:10E4F000A3E0FA1609F043C080910E03813009F0C1
:10E500003EC07091530260E080915202680F711D0D
:10E51000709327046093260488E090E040E750EF72
:10E520000E9451F5E199FECF1FBA1EBA8FEF8DBB45
:10E530000FB6F894E29AE19A0FBEE199FECF81E01E
:10E5400090E09FBB8EBB8FEF8DBB0FB6F894E29A25
:10E55000E19A0FBE10922D0410922E0410922F04F7
:10E560001092300480E090E0A0E0BFEF80930F03B2
:10E5700090931003A0931103B093120391E0809144
:10E580005102853021F580910E03813009F06BC076
:10E590008091520290915302A0915402B091550281
:10E5A0008093140390931503A0931603B09317035D
:10E5B00090E0E92FF0E0DF01A35BBD4F1B968C914B
:10E5C000EC5EFC4F84839F5F903899F74BC0863098
:10E5D00009F049C080910E03813009F044C090E0F9
:10E5E000E92FF0E0DF01A35BBD4F1B968C91E8564D
:10E5F000FC4F80839F5F903899F70E9441F12091F2
:10E60000290430912A0440912B0450912C0420308D
:10E61000B0EF3B07B1E04B07B0E05B0710F090E0D4
:10E6200022C080910F0390911003A0911103B0912B
:10E63000120382179307A407B50721F0CA01B90195
:10E640000E949DF18091290490912A04A0912B04AD
:10E65000B0912C0480930F0390931003A0931103A7
:10E66000B093120391E080915102893009F058C0B3
:10E6700080910E03813009F053C0209152023091F5
:10E680005302409154025091550280912D04909173
:10E690002E04A0912F04B0913004281739074A079F
:10E6A0005B0711F090E03CC0E199FECF1FBA1EBAA3
:10E6B00081E08DBB0FB6F894E29AE19A0FBE2091EB
:10E6C0002604309127048DB79EB708970FB6F894AB
:10E6D0009EBF0FBE8DBFEDB7FEB731960AEF12E0B9
:10E6E000ADB7BEB712961C930E93119780E091E0E0
:10E6F00093838283348315823070378326830E940C
:10E7000066F58DB79EB708960FB6F8949EBF0FBEFC
:10E710008DBF80E40E940AF5C8010E940EF591E0C9
:10E720008AE28093E602E092E702D092E80283E078
:10E730008093E90284E68093EA02F092EB029093E0
:10E74000EC020E941FF11F910F91FF90EF90DF905C
:10E7500008951F93CF93DF93A8952FE088E190E071
:10E760000FB6F894A89581BD0FBE21BD10929800F8
:10E7700083E28093990088E180939A0080916400FD
:10E78000816080936400119A189A8B9A929A0E94E1
:10E79000C6F40E9402F580E00E940AF5E199FECFDE
:10E7A00082E090E09FBB8EBBE09A8DB38F3F11F467
:10E7B0000E94E8F184E090E068E670EF0E943BF58B
:10E7C000909332048093310486E090E068E670EF25
:10E7D0000E943BF5909348018093470188E090E0C8
:10E7E00068E670EF0E943BF590932704809326041F
:10E7F000E199FECF8AE090E09FBB8EBBE09A8DB39B
:10E8000081E08093E502CAEFD2E0CE0164E171E0DD
:10E810000E9434F5CE010E940EF580E40E940AF5B4
:10E8200020912604309127048DB79EB708970FB624
:10E83000F8949EBF0FBE8DBFEDB7FEB73196ADB752
:10E84000BEB71296DC93CE93119785E291E0938345
:10E850008283348315823070378326830E9466F565
:10E860008DB79EB708960FB6F8949EBF0FBE8DBFAA
:10E870008091260490912704892B29F4CE0169E325
:10E8800071E00E9434F58AEF92E00E940EF585E077
:10E8900083BF8BE08EBD80E893E49BBD8ABD16E00C
:10E8A000A89506B604FE05C086B7806186BF0E94A3
:10E8B0008AF080919B0087FF02C00E94C7F0809180
:10E8C0009B0086FF1BC080919B00806480939B000F
:10E8D0009091460180912504981710F00CC0A895DE
:10E8E00080919B0085FFFBCFE92FF0E0EA51FD4FBF
:10E8F000808180939C009F5F9093460180912404C7
:10E90000882321F00E941CF2109224048091330489
:10E910008450823028F6109333048CB390E0FC01CD
:10E92000E270F07081FDF9CF1FBA1EBAE09A8DB384
:10E93000813009F0B5CF0995B3CF9FEF97BB88BB66
:10E940001E981B9A1F9A83E0982F9A95F1F71F98AB
:10E9500017BA1E9A1B981F9A8A95F1F7B799FECF9E
:10E960001F9808959FEF97BB88BB1E981B981F9A0E
:10E9700083E0982F9A95F1F71F9817BA1E9A1F9A5D
:10E980008A95F1F7B799FECF1F9808958FEF87BB4F
:10E99000169A139A179A18BA1E981B981F9880E314
:10E9A00088BB1F9A22E1922F9A95F1F71F98ECEC01
:10E9B000FAE03197F1F788BB1F9A922F9A95F1F7F9
:10E9C0001F9898EB392F3A95F1F788BB1F9A822F41
:10E9D0008A95F1F71F98892F8A95F1F788E388BB0C
:10E9E0001F9A822F8A95F1F71F989A95F1F78CE07C
:10E9F00088BB1F9A2A95F1F71F9889E995E101973D
:10EA0000F1F7089581E00E94B2F4089582E00E9437
:10EA1000B2F4089580580E94B2F40895CF93DF9322
:10EA2000EC0103C00E949DF4219688818823D1F7D0
:10EA3000DF91CF910895CF92DF92EF92FF921F93D3
:10EA40006B017C0110E003C00E949DF41F5FE12F69
:10EA5000F0E0EC0DFD1D84918823B1F71F91FF902C
:10EA6000EF90DF90CF900895FB01DC0101900D92B3
:10EA70000020E1F70895DF92EF92FF920F931F932A
:10EA80007B018C01FB010995D82EC8010196F70185
:10EA90000995982F8D2D1F910F91FF90EF90DF908A
:10EAA0000895DF92EF92FF920F931F93D72E7A0172
:10EAB0008C01FA010995C80101966D2DF7010995A0
:10EAC0001F910F91FF90EF90DF900895AEE0B0E0BE
:10EAD000ECE6F5EF0C9429F80D891E8986E08C830D
:10EAE0001A8309838FEF9FE79E838D839E01275EA4
:10EAF0003F4FCE0101966F89788DA9010E948AF55A
:10EB00002F813885020F131FF80110822E96E4E042
:10EB10000C9445F8ABE0B0E0E0E9F5EF0C941BF89D
:10EB20003C012B015A01FC0117821682838181FD71
:10EB300003C06FEF7FEFC6C19AE0892E1E010894D3
:10EB4000211C311CF3012381F20123FD859123FF58
:10EB500081912F01882309F4B2C1853239F423FD54
:10EB6000859123FF81912F01853229F490E0B30133
:10EB70000E947DF7E7CF982FFF24EE249924FFE130
:10EB8000FF15D0F09B3269F09C3228F4903259F096
:10EB9000933291F40EC09D3249F0903369F441E014
:10EBA00024C052E0F52A84E0F82A28C098E0F92A27
:10EBB00025C0E0E1FE2A22C0F7FC29C0892F80533E
:10EBC0008A3070F4F6FE05C0989C902C1124980EA3
:10EBD00015C0E89CE02C1124E80EF0E2FF2A0EC0DC
:10EBE0009E3229F4F6FC6BC140E4F42A07C09C363F
:10EBF00019F450E8F52A02C0983649F4F20123FDD1
:10EC0000959123FF91912F01992309F0B8CF892F76
:10EC10008554833018F08052833038F444E050E05B
:10EC2000A40EB51E5FE359830FC0933631F09337BE
:10EC300079F0933509F056C020C0F50180818983B1
:10EC400042E050E0A40EB51E610101E010E012C0E8
:10EC5000F501C080D180F6FC03C06FEF7FEF02C0EA
:10EC6000692D70E042E050E0A40EB51EC6010E947E
:10EC700072F78C015FE7F52214C0F501C080D180E6
:10EC8000F6FC03C06FEF7FEF02C0692D70E042E039
:10EC900050E0A40EB51EC6010E9467F78C0150E833
:10ECA000F52AF3FE07C01AC080E290E0B3010E948B
:10ECB0007DF7EA948E2D90E008171907A8F30EC08F
:10ECC000F601F7FC8591F7FE81916F0190E0B301A9
:10ECD0000E947DF7E110EA940150104001151105E2
:10ECE00079F7EAC0943611F0993669F5F7FE08C055
:10ECF000F501208131814281538184E090E00AC096
:10ED0000F501808191819C01442737FD4095542F66
:10ED100082E090E0A80EB91E9FE6F92257FF09C0D5
:10ED200050954095309521953F4F4F4F5F4FE0E80C
:10ED3000FE2ACA01B901A1012AE030E00E94A9F728
:10ED4000D82ED21840C0953729F41F2D1F7E2AE0F7
:10ED500030E01DC01F2D197F9F3661F0903720F4E1
:10ED6000983509F0ACC00FC0903739F0983709F0EA
:10ED7000A6C004C028E030E00AC0106114FD146091
:10ED800020E130E004C014FD166020E132E017FFFE
:10ED900008C0F501608171818281938144E050E077
:10EDA00008C0F50180819181BC0180E090E042E0E3
:10EDB00050E0A40EB51EA1010E94A9F7D82ED218CA
:10EDC0008FE7F82EF122F6FE0BC05EEFF522D91484
:10EDD00038F4F4FE07C0F2FC05C08FEEF82202C042
:10EDE0001D2D01C0192DF4FE0DC0FE01ED0DF11D0C
:10EDF0008081803319F499EEF92208C01F5FF2FE7A
:10EE000005C003C08F2D867809F01F5F0F2DF3FC1E
:10EE100014C0F0FE0FC01E1510F09D2C0BC09D2CD1
:10EE20009E0C911A1E2D06C080E290E0B3010E9454
:10EE30007DF71F5F1E15C0F304C01E1510F4E11A04
:10EE400001C0EE2404FF0FC080E390E0B3010E94F4
:10EE50007DF702FF1DC001FD03C088E790E00EC0F2
:10EE600088E590E00BC0802F867891F001FF02C00A
:10EE70008BE201C080E2F7FC8DE290E0B3010E94DA
:10EE80007DF706C080E390E0B3010E947DF79A947D
:10EE9000D914C0F3DA94F101ED0DF11D808190E0F9
:10EEA000B3010E947DF7DD20A9F706C080E290E063
:10EEB000B3010E947DF7EA94EE20C1F743CEF3013F
:10EEC00066817781CB012B96E2E10C9437F8FC0147
:10EED0000590615070400110D8F7809590958E0F85
:10EEE0009F1F0895FC016150704001900110D8F7F8
:10EEF000809590958E0F9F1F08950F931F93CF932A
:10EF0000DF938C01EB018B8181FF1BC082FF0DC061
:10EF10002E813F818C819D812817390764F4E88117
:10EF2000F9810193F983E88306C0E885F985802F8C
:10EF30000995892B31F48E819F8101969F838E8361
:10EF400002C00FEF1FEFC801DF91CF911F910F910A
:10EF50000895FA01AA27283051F1203181F1E8946F
:10EF60006F936E7F6E5F7F4F8F4F9F4FAF4FB1E0BC
:10EF70003ED0B4E03CD0670F781F891F9A1FA11DB7
:10EF8000680F791F8A1F911DA11D6A0F711D811DB8
:10EF9000911DA11D20D009F468943F912AE0269F7D
:10EFA00011243019305D3193DEF6CF010895462FDC
:10EFB0004770405D4193B3E00FD0C9F7F6CF462FBD
:10EFC0004F70405D4A3318F0495D31FD4052419326
:10EFD00002D0A9F7EACFB4E0A695979587957795E3
:10EFE0006795BA95C9F700976105710508959B016A
:10EFF000AC010A2E06945795479537952795BA95F3
:10F00000C9F7620F731F841F951FA01D0895AA1BC7
:10F01000BB1B51E107C0AA1FBB1FA617B70710F003
:10F02000A61BB70B881F991F5A95A9F78095909535
:10F03000BC01CD0108952F923F924F925F926F9243
:10F040007F928F929F92AF92BF92CF92DF92EF9278
:10F05000FF920F931F93CF93DF93CDB7DEB7CA1BF9
:10F06000DB0B0FB6F894DEBF0FBECDBF09942A8824
:10F07000398848885F846E847D848C849B84AA84CC
:10F08000B984C884DF80EE80FD800C811B81AA8159
:10F09000B981CE0FD11D0FB6F894DEBF0FBECDBF24
:08F0A000ED010895F894FFCF83
:10F0A8004669726D776172652025692E253032694F
:10F0B800204F4B004C6472264677206279204F4BD4
:10F0C8003254505100426F6F74696E672E2E2E2095
:10F0D8007625692E25303269004E6F206669726D7B
:06F0E80077617265000073
:040000031000E00009
:00000001FF
